:100000000000000000002A28A301A200FF30A20780
:10001000031CA307031C26280330A100DF30122095
:100020000628A101E83EA000A109FC30031C1B2802
:10003000A00703181828A0070000A10F18282018EF
:100040002128A01C252800002528080083138312DE
:1000500003130800830183168117063083129F0063
:100060000730831685008601C83083120420051EE0
:100070004E28851940280130A500F430A4004328FB
:10008000A501C830A40086152508A3002408052072
:1000900086112508A300240805203728861537284F
:0200A0005028E6
:02400E00981EFA
:00000001FF
